S123D0007ED1AC0D0A043E3E20045155495404434154414C4F4720045341564520044C4F02
S123D0204144200452554E200444454C45544520044154545249425554452004494E464F4F
S123D04020044E414D452004464F524D415420044552524F5220044F4B0D0A044E4F205303
S123D06050414345204C4546540D0A0446494C45204E4F5420464F554E440D0A044C4F4169
S123D08044494E470D0A0444454E4945440D0A042053544152543A0420454E443A044E41DB
S123D0A04D452020202020202020202020202020202020202020415454522020204C4F41E3
S123D0C0442020202020202053495A450D0A045459504520275945532720544F20434F4E6E
S123D0E04649524D0D0A040D0A464F524D415454494E470D0A0448454C500D0A20202020F6
S123D100515549434B46494C4520312E300D0A2020202043202D20434154414C4F470D0A66
S123D1202020202053202D20534156450D0A202020204C202D204C4F41440D0A2020202075
S123D14052202D2052554E204C4F41440D0A2020202044202D2044454C4554450D0A202085
S123D16020204E202D204E414D450D0A2020202041202D204154545249425554450D0A205F
S123D18020202049202D20494E464F0D0A2020202046202D20464F524D41540D0A202020BF
S123D1A02051202D20515549540D0A0496029780840F8100260486879780868097027F0000
S123D1C0857F00867F00877F0088BDD955BDD97A24037ED26A86ECB78067CE7C00BDD99B4D
S123D1E0BDD97A24037ED26AB67C7B9781B67C7A9782B67C799783B67C789784CED003BDC8
S123D200C0097F00A3CED006BDC009BD7FEB84DF815126037ED26D814326037ED27A815328
S123D22026037ED330814C26037ED405815226037ED3FC814426037ED4AC814126037ED580
S123D2401A814926037ED5C1814E26037ED640814626037ED6C0814826037ED77E863FBDD2
S123D260C003CED003BDC00920987EC00096809702CED00ABDC0097EC000CED00FBDC0097C
S123D280BDD787CE0089BDD7E825037ED327CED003BDC0097F00857F00867F00877F0088BF
S123D2A0BD7FE5810027037ED322BDDA0B8601B780628620B78067CE7C00BDD99BBDD97A9A
S123D2C024037ED31FBDD919243EB67C0B81012637B67C0C81012630968981002705BDD80F
S123D2E04724258620BDC003BDC003BDC003BDC003CE7C0FBDD7CE8620BDC003BDC003BDD6
S123D300D793CED003BDC009DE8508DF859681918527037ED2A09682918627037ED2A07E9B
S123D320D202BD7FEB20F8CED003BDC0097ED202CED018BDC009BDD8BF250FCED003BDC07B
S123D34009CED05CBDC0097ED202BDD90DCE7C0FBDD7E825037ED3A0B67C0F8100274186AD
S123D36001B77C0B8601B77C0C8607B77C2ECED090BDC009BDC01E2427FF7C2FCED098BD7F
S123D380C009BDC01E2419DFA1CED003BDC009B67C2F4C4C7C7C0E7C7C3291A123F420129D
S123D3A0CED003BDC0097ED202CED05CBDC0097ED202CE0001DF87BDDA0BB67C32B780624A
S123D3C08630B78067FE7C2FBDD9EEBDD970BDD97A25CDCE0000DF87BDDA0B8601B78062CA
S123D3E08630B78067CE7C00BDD9D3BDD970BDD97A25ADCED057BDC0097ED202CED024BDEE
S123D400C0097C00A3CED01EBDC009BDD787CE0089BDD7E8241A968981002714CED003BD79
S123D420C009BDD865251BCED06CBDC0097ED202CED003BDC0097ED202CED087BDC0097E61
S123D440D202B67C2E840127F0CED07DBDC009CE0001DF87BDDA0BB67C32B780628620B726
S123D4608067FE7C2FBDD9B6BDD97A24037ED43009DFA1CE7C2FBDC0158608BDC003862DBE
S123D480BDC003CE00A1BDC015CED003BDC0097D00A32609CED057BDC0097ED202B67C2E64
S123D4A084042795BDDA24FE7C2F6E00CED029BDC009BDD787CE0089BDD7E8241A96898139
S123D4C0002714CED003BDC009BDD865251BCED06CBDC0097ED202CED003BDC0097ED20251
S123D4E0CED087BDC0097ED202B67C2E840227F0BDD90D7F7C0BBDDA0B8601B7806286300D
S123D500B78067CE7C00BDD9D3BDD970BDD97A25C6CED057BDC0097ED202CED031BDC00993
S123D520BDD787CE0089BDD7E8241A968981002714CED003BDC009BDD8652512CED06CBDC1
S123D540C0097ED202CED003BDC0097ED202860DBDC003BDD793BD7FEB84DF8152271581DF
S123D56057271B81582721810D2727CED003BDC0097ED202B67C2E8801B77C2E20D0B67C2C
S123D5802E8802B77C2E20C6B67C2E8804B77C2E20BCCED003BDC009CE0000DF87BDDA0B62
S123D5A08601B780628630B78067CE7C00BDD9D3BDD970BDD97A258DCED057BDC0097ED2AD
S123D5C002CED03CBDC009BDD787CE0089BDD7E8241A968981002714CED003BDC009BDD822
S123D5E0652512CED06CBDC0097ED202CED003BDC0097ED202CED09EBDC009CE7C0FBDD781
S123D600CEBDD7938620BDC003BDC003CE7C2FBDC0158608BDC003862DBDC003BDD940DF6A
S123D620A1CE00A1BDC0158620BDC003CE7C0DBDC0158620BDC003CED003BDC0097ED20296
S123D640CED042BDC009BDD787CE0089BDD7E8241A968981002714CED003BDC009BDD86538
S123D6602512CED06CBDC0097ED202CED003BDC0097ED2028620BDC003BDC003BDC003BD31
S123D680C003BDC003BDC003BDC003BDC003CE7C0FBDD7E824D5CED003BDC009BDDA0B86A6
S123D6A001B780628630B78067CE7C00BDD9D3BDD970BDD97A25B4CED057BDC0097ED20209
S123D6C0CED048BDC009BD7FEB810D27037ED775CED003BDC009CED0CFBDC009BDC0068113
S123D6E05927037ED775BDC006814527037ED775BDC006815327037ED775CED0E7BDC00946
S123D7007F00857F00867F00877F0088BDDA31864DB77C008643B77C018646B77C0286534A
S123D720B77C038601B77C04CE0085BDC015DE85FF7C05CEFFFFFF7C09BDDA0B8601B78079
S123D74062BDD9708630B78067CE7C00BDD9D3BDD970BDD97A251EDE8508DF859681918501
S123D7602606968291862707860DBDC00320B9CED057BDC009CED003BDC0097ED202CED09E
S123D780F6BDC0097ED202CE00896F00088C00A126F839862DF67C2EC401C101260286528B
S123D7A0BDC0038620BDC003862DF67C2EC402C10226028657BDC0038620BDC003862DF68F
S123D7C07C2EC404C10426028658BDC0033936375FA600810026028620BDC003085CC118D1
S123D7E027037ED7D133323936375FA6008100270BBDC003085CC118220220EFBD7FEB817A
S123D8001B2740817F27F522F38108270B810D272E811F23E77ED831C10027E0095ABDC0DA
S123D820038620BDC0038608BDC0034FA7007ED7FCC11827C7BDC003A700085C7ED7FC3390
S123D840320D3933320C395FC1182715CE00893AA600812A270BCE7C0F3AA10026055C203F
S123D860E70D390C397F00857F00867F00877F0088BDDA0B8601B780628620B78067CE7CCC
S123D88000BDD99BBDD97A24037ED8BBBDD9192413B67C0B8101260CB67C0C81012605BD8C
S123D8A0D8472519DE8508DF859681918527037ED8719682918627037ED8710C390D397FF0
S123D8C000857F00867F00877F0088BDDA0B8601B780628620B78067CE7C00BDD99BBDD996
S123D8E07A24037ED909BDD9192407B67C0B81002719DE8508DF859681918527037ED8CB04
S123D9009682918627037ED8CB0C390D39CE7C0C6F00088C7D9026F839B67C00814D261EFD
S123D920B67C0181432617B67C0281462610B67C0381532609B67C04810126020D390C39DB
S123D940FE7C2FB67C32C6FF810027073A083A084A20F509398604B78067BDD97086E0B7D2
S123D96080668601B7806186EFB78067BDD97039B680678480810026F739B6806784018131
S123D9800027163CCED050BDC009FE8061BDC012CED003BDC009380D390C39BDD970BDD9A2
S123D9A07AB68067840881082608B68060A7000820E9BDD97039BDD970BDD97AB680678445
S123D9C008810826EDB68060BDDA24A700BDDA240820E3BDD970BDD97AB680678408810819
S123D9E02608A600B780600820E9BDD97039BDD970BDD97AB680678408810826EDBDDA24D2
S123DA00A600BDDA24B780600820E39688B780639687B780649686B780659685840F8AE0BF
S120DA20B780663936379602D680D7029780333239CE7C006F00088C7E0026F83904
S9030000FC
